:04000000B601FA2823
:1000080008000408A7008810081008108316881034
:10001800081008100F30880583122708B6183228F0
:100028003A30A1009830A2203330A6004620133081
:10003800A1008830A22046206430A12046206430E8
:10004800A1202230A6004620283031200C30312053
:1000580006303120B614270832283614A600361C7C
:1000680040280810033C031C452845200730A10000
:10007800D030A220031408003614FE3C0319F528DA
:100088000814361C361088140F3088052608F039F5
:1000980088048810A60E361846283230A12003148A
:1000A8000800B71329080319B7170530A800273027
:1000B800A30010306B200330A300E8306B20A301AD
:1000C80064306B20A3010A306B2024087228A20038
:1000D8002508A1002408A000D4202008A000A80317
:1000E8000319B713290803197C28280203180800E4
:1000F8002008031DB713B71B0800303EF028A000E6
:10010800A00DA00D200D3839C1389F000030A10086
:100118001430A2201F151F198F28A1011E08F528C9
:10012800A301A200FF30A207031CA307031CF528A4
:100138000330A100DF30A2209628A101E83EA000EC
:10014800A109FC30031CAB28A0070318A828A007A6
:100158006400A10FA8282018B128A01CB528000009
:10016800B5280800A101A301A2000230BD28A20001
:100178000530A80023082102031DC42822082002F4
:10018800043003180130031902302805031DFF301D
:10019800F5280038031DFF300405031DFF30F5283E
:1001A800A501A4011030A600210DA40DA50D22085B
:1001B800A4022308031C230FA5020318EA28220817
:1001C800A40723080318230FA5070310A00DA10DEA
:1001D800A60BD8282008F528840031088A003008A2
:1001E8008200831303138312640008000811831626
:1001F800081183120130A300F4308A019520BD0153
:10020800C001C201BF01831607308900FF30850095
:100218001F3086008312860183169F0183120130E6
:10022800C4008316553081008312A0308B008B17D1
:100238008A110A1224298B1B08008A110A12152B0D
:100248008A011F21003006180130A00001308A0100
:10025800B620B2000030061A0130A00001308A0131
:10026800B620B4003208840034088A01CD208A11EF
:100278000A12031DD12A8A011F21003006180130F5
:10028800A00001308A01B620B20000308619013082
:10029800A00001308A01B620B40032088400340876
:1002A8008A01CD208A110A12031DA52A8A011F215D
:1002B800003006180130A00001308A01B620B200D3
:1002C800003006190130A00001308A01B620B400C0
:1002D8003208840034088A01CD208A110A12031DCD
:1002E800E82A8A011F21003006180130A0000130D9
:1002F8008A01B620B200003086180130A000013013
:100308008A01B620B4003208840034088A01CD205E
:100318008A110A12031DBB2A8A011F2100308A0193
:100328008320C1008A011F214108A000A1010530D6
:10033800A200A3018A01D420C1008A011F21640000
:100348004408013C8A110A12031D5D2A8A011F21F3
:10035800FE308A01062002308A0106208A011F2108
:100368003D08BC008A011F213D08A000A1010C30F6
:10037800A200A3018A01D4202408B2002508B300F2
:100388003208A0003308A100A30100308A01BB2075
:100398008A110A12031DD6298A011F210C30BC07B5
:1003A8008A011F218A011F2164000C303D028A1135
:1003B8000A120318192A8A011F2120308A010620EF
:1003C80020308A01062053308A01062048308A01ED
:1003D800062020308A0106200230A9003C08A4002B
:1003E800A5010530B000B1018A0155203A308A01D3
:1003F80006200230A9003F08A400A5010530B0007E
:10040800B1018A0155203A308A0106200230A9003C
:100418004008A400A5010530B000B1018A015520AB
:100428008A011F218A110A12582A8A011F212030A5
:100438008A01062020308A0106204F308A010620D2
:1004480053308A01062020308A0106200230A90094
:10045800F4303C07B200FF300318013EB300320805
:10046800A4003308A5000530B000B1018A01552069
:100478003A308A0106200230A9003F08A400A501ED
:100488000530B000B1018A0155203A308A010620B2
:100498000230A9004008A400A5010530B000B10150
:1004A8008A0155208A011F218A011F21C4018A015E
:1004B8001F218A011F21FE308A010620C0308A01CF
:1004C80006200230A900FF304107B200FF300318B0
:1004D800013EB3003208A4003308A5000530B0007F
:1004E800B1018A01552020308A01062043308A0153
:1004F800062020308A01062020308A01062020307C
:100508008A01062032308A01062030308A0106200E
:1005180030308A01062033308A0106202F308A01C4
:10052800062068308A0106207A308A010620723057
:100538008A0106206E308A0106208A011F218A015D
:1005480024298A011F21BF0A8A011F2164003C3027
:100558003F028A110A12031CB62A8A011F21BF0111
:100568008A011F218A011F218A110A12FA2A8A0187
:100578001F21BD0A8A011F21640018303D028A111B
:100588000A12031CCC2A8A011F21BD018A011F21DE
:100598008A011F218A110A12FA2A8A011F21BF0320
:1005A8008A011F2164003C303F028A110A12031C91
:1005B800E32A8A011F213B30BF008A011F218A01DB
:1005C8001F218A110A12FA2A8A011F21BD038A01F2
:1005D8001F21640018303D028A110A12031CFA2AEE
:1005E8008A011F211730BD008A011F218A011F219E
:1005F8000F308A0194208A011F210130C4008A012A
:100608001F211F300605C3008A011F21640043080B
:10061800013C8A110A120319A1298A011F218A01A2
:10062800FA2AC20A64003D3042028A110A12031CE7
:100638003B2BC201C00A64003C3040028A110A12F6
:10064800031C392BC001BF0A64003C303F028A11E9
:100658000A12031C392BBF01BD0A640018303D0281
:100668008A110A12031C392BBD010130C400A030C5
:0E0678008B0009008A011F2163008A01402BBC
:02400E00713D02
:00000001FF
